:040000000C946A00F2
:100004000C9400000C9400000C9400000C9400006C
:100014000C9400000C9400000C9400000C9400005C
:100024000C9400000C9400000C9400000C9400004C
:100034000C9400000C9400000C9400000C94CC0070
:100044000C9400000C9499000C9400000C94000093
:100054000C9400000C9400000C9400000C9400001C
:100064000C9400001027E80364000A00010000104B
:10007400000110000100000000000A000000000060
:10008400000000000000000000000000000000006C
:10009400000000000000000000000000000000005C
:1000A4000000000000000000000000000A0A0A0A24
:1000B4000A0A0A0A0A0A0A0A0A0A0A0A02000200C0
:1000C4007A00020004007C00010008037E000000A6
:1000D400F894EE27EFBBF1E0F5BFE5BF8DE0A2E0B9
:1000E400BB27ED938A95E9F780E098E0A0E0B1E0C2
:1000F400ED930197E9F7E0ECF0E085919591009795
:1001040061F0A591B59105901590BF01F00105909E
:100114000D920197E1F7FB01F0CFE8E0EEBBEFEFC2
:10012400EDBFE8E0EEBFC0E0D3E00C94A203AA93D5
:10013400EA93FA93EFB7EA931A930A931091C000E3
:100144000091C600E12FEC71E9F4E091F403EF5F54
:10015400E093F403E150F0E0E552FC4F0083A091FA
:10016400F403A93119F4E0E0E093F403A091F60359
:10017400AF5FA093F603A93129F4E0E0E093F6031E
:10018400689437F809911991E991EFBFF991E991D0
:10019400A99118950A921A926A937A938A939A93D8
:1001A400AA93BA93EA93FA93EFB7EA93E0913B03E5
:1001B400F0913C033196E0933B03F0933C030E949F
:1001C4001522E1E5F1E00E945A2C0E2E0E94152220
:1001D400E3EAF2E00E945A2CE02909F416C2A09145
:1001E4003903B0913A03E4E1F0E00E946C2C0E2E46
:1001F400E0910503F0E074970E94602C0E22A09118
:100204002003EEE00E94502CE02121F0E091200335
:10021400EF5F03C025FC03C0E0E0E0932003A0915E
:100224002003AE3011F4689425F8E0913903E0938B
:100234000503A0912903A13029F4F79B02C0F79884
:1002440001C0F79AE1E02E260E941A220E9423227E
:10025400E093BF03F093C0036093C1037093C203A0
:100264000E942A22A3EAB3E00E942F220E9436228F
:10027400AFECB3E00E942F220E943B220E94442252
:100284000E94862BE093A303F093A4036093A50339
:100294007093A603A091CF03B091D0038091D103B2
:1002A4009091D203E0E0F0E060E772E40E94862BD4
:1002B400E093CF03F093D0036093D1037093D20300
:1002C4000E9449220E944E220E2E0E9453220E9416
:1002D4004E22E02161F1E091CF03F091D0036091CF
:1002E400D1037091D2030E943B220E94862BE0939B
:1002F400CB03F093CC036093CD037093CE030E94A1
:100304005822ADE4B3E00E946122A091CB03B091E6
:10031400CC038091CD039091CE030E942322E093DD
:10032400AB03F093AC036093AD037093AE030E94F0
:1003340066220E9477220E94E82AE093B303F09396
:10034400B4036093B5037093B6030E9466220E94BF
:1003540080220E94E82AE093D703F093D8036093A5
:10036400D9037093DA030E9489220E9492220E9488
:10037400A522ABE8B3E00E94772A0E944E2D0E948A
:100384008922AAE0B0E080E090E00E94922C0E94D2
:1003940080220E94AC2A0E94CB2B70F0E0E0E09314
:1003A400D703E093D803E093D903E093DA030E94E0
:1003B400AA2231960E94AF22E0918F03F09190031C
:1003C4006091910370919203A091B703B091B80327
:1003D4008091B9039091BA030E94382BDF01CB01BD
:1003E4000E942322E093C303F093C4036093C503E4
:1003F4007093C6030E94B4220E94E82A0E94BD2280
:10040400E0910F03F0E00E94C6220E942D2C0E946E
:10041400CF22ADE6B3E00E94DE220E941A220E949F
:10042400AE2D3CF5A091C303B091C4038091C503E4
:100434009091C6030E94E3227F936F93FF93EF93FF
:10044400A091BF03B091C0038091C1039091C203F6
:100454000E94E322AF91BF918F919F910E94862BBE
:10046400E093BB03F093BC036093BD037093BE039E
:1004740009C0E0E0E093BB03E093BC03E093BD0359
:10048400E093BE03A091BE03AA238AF40E94EA2249
:100494000E94F32218F40E94FA2208C00E94012349
:1004A4000E94422AA5E7B3E00E94DE2214C00E9403
:1004B400EA22E0E0F0EC69E774E40E94CB2B09F057
:1004C40008F403C00E94FA2206C00E940123A5E793
:1004D400B3E00E94DE220E940A230E9413230E949A
:1004E400E82A0E941C23E091A303F091A4036091E5
:1004F400A5037091A6030E9425230E94CB2B68F5C7
:10050400E091AB03F091AC036091AD037091AE0345
:100514000E9425230E94E82AE093A703F093A803EE
:100524006093A9037093AA030E9425230E942E239B
:100534000E94E12ADF01CB010E9458220E94862BEF
:10054400A0E0B0E081E695E40E94382BA9E6B3E090
:100554000E94DE22689424F802C0E0E12E260E9464
:100564000A230E9437230E94E82AE093AF03F09302
:10057400B0036093B1037093B2030E943723E0E0A9
:10058400F0E060E87FE30E94CB2B09F008F412C08E
:10059400E093AF03E093B003E093B103E093B203BD
:1005A4000E944023EF5FFF4F6F4F7F4F0E9449230C
:1005B4000E9452230E945823A034E2E4BE07EFE0D5
:1005C4008E07E0E09E0778F0E0E0E0935B03E093C1
:1005D4005C03E0935D03E0935E03AFE3B0E00E944D
:1005E40061230E94832D0E9413230E946623ADE39E
:1005F400B3E00E946122A0911E03AC3308F4F29888
:10060400A0911E03AC3309F4F29A0E941522A33A76
:10061400E2E0BE0709F06BC0A0911D030E946A23AB
:100624000E946F230E9461230E94722C0E947823EF
:10063400E02191F0E0911E03EF5FE0931E03E0914F
:100644001D03F0E03296A0911E03B0E0EA17FB0709
:1006540019F4ECE3E0931E03E0E0E0933B03E09342
:100664003C03D394A0911003A13028F4E09110032B
:10067400EF5FE09310030E947F23E8E5F2E00E941D
:10068400662C0E2E0E948423E021E9F0E0915103B0
:10069400F09152033196E0935103F09352030E9478
:1006A4007F230E948923EA1BFB0BE0935703F093FB
:1006B40058030E946F230E94AE2D2CF4E0E0E093D7
:1006C4005103E0935203ECE3ED1589F4DD24C39464
:1006D400EC1569F4CC24E0910003EF5FE093000390
:1006E400A0910003A43119F4E0E0E0930003E99140
:1006F400EFBFF991E991B991A99199918991799172
:100704006991199009901895AA93E881E066E0939D
:100714007C0085E28A95F1F7E0917A00E064E09349
:100724007A00E0917A00E071E1F3E0917A00E0610F
:10073400E0937A00E0917800F09179002196089591
:10074400EF97279780E4A6E0B0E0E0E8F0E00E94AD
:10075400C32DFF2401E021E0E0E8E0936100E0E044
:10076400E0936100EFE0E4B9E1E0E5B9E0E0E7B986
:10077400E4E0E8B9EAEFEAB9E7EEEBB9E0E0E4BDBA
:10078400E3E0E5BDE0E0E6BDE7BDE8BDE093800061
:10079400E0938100E0938500E0938400E093870078
:1007A400E0938600E0938900E0938800E0938B0057
:1007B400E0938A00E093B600E1EAE093B000E2E05F
:1007C400E093B100E0E0E093B200E093B300E09383
:1007D400B400E1E0E0936E00E0E0E0936F00E093AA
:1007E4007000E0936900EDBBE0936800E093C00003
:1007F400E8E9E093C100E6E0E093C200E0E0E093C2
:10080400C500E7E4E093C400E0E8E0BFE0E0E09383
:100814007F00E0937E00E0E6E0937C00E6E2E09374
:100824007A00E0E0E0937B00ECBDE093BC007894B8
:100834005F9A0E948E230E9492230E949F230E940B
:10084400AC230E948E23EAE06E1668F4ADE2B0E0B9
:100854000E94B923A8E2B0E0E0E00E94932DA9E24F
:10086400B0E00E94932DEAE09E1650F4A3E3B0E0BA
:100874000E94B923ABE3B0E00E94B923689426F840
:10088400EAE0BE1618F4689430F827F8689433F850
:10089400E6E1E09312030E94BE230E94C5230E9456
:1008A400CC23E8ECF0E0E0936303F0936403A0E06E
:1008B400B0E00E94772DE0931303A1E0B0E00E9422
:1008C400772DE0931403A2E0B0E00E94772DE0932B
:1008D4001503A3E0B0E00E94772DE0931703A4E092
:1008E400B0E00E94772DEC8FA5E0B0E00E94772D58
:1008F400ED8FA6E0B0E00E94772DEE8FA7E0B0E088
:100904000E94772DE0931803A8E0B0E00E94772DB1
:10091400E0931903A9E0B0E00E94772DE0931A0355
:10092400F798F198AAE0B0E00E94772DE0931D03B8
:10093400ABE2B0E00E94732D0E94D323A4E1B0E0A7
:100944000E94772DE88FA5E1B0E00E94772DE98F12
:10095400A6E1B0E00E94772DEA8FABE0B0E00E9400
:10096400772DEC8BACE0B0E00E94772DED8BADE001
:10097400B0E00E94772DEE8BAFE2B0E00E94732DC1
:10098400EB87FC87AEE0B0E00E94772DE0932A036A
:10099400AFE0B0E00E94772DE0932C03A0E1B0E03B
:1009A4000E94772DE0932B03AFE3B0E00E946F2DFC
:1009B4000E944923ADE2B0E00E94732DAFE9B3E099
:1009C4000E94D8230E942E23ADE3B3E00E9461224B
:1009D4000E9413230E94DF230E941C23A1E1B0E0A4
:1009E4000E94772D3E2FA1E3B0E00E94732DEF8784
:1009F400F88BA2E1B0E00E94772DE8A3A3E1B0E078
:100A04000E94772DEF8FA3E3B0E00E94732DA3EB38
:100A1400B3E00E94D823ABE3B0E00E94732DA3EDB2
:100A2400B3E00E94D8230E94B4220E94DF230E94D4
:100A3400BD22A5E3B0E00E94732D0E94E323A9E345
:100A4400B0E00E94732D0E942D2C0E94E823A7E1A0
:100A5400B0E00E94772D0E94BE2D23F8A7E3B0E0FA
:100A64000E94732D0E94F123A8E1B0E00E94772D2B
:100A7400E0930703A9E1B0E00E94772DE093090316
:100A8400AAE1B0E00E94772DE0930A03ABE1B0E065
:100A94000E94772DE0930B03ACE1B0E00E94772D28
:100AA400E0930C03ADE1B0E00E94772DE0930D03D9
:100AB400AEE1B0E00E94772DE0932103AFE1B0E016
:100AC4000E94772DE0932203A0E2B0E00E94772DEC
:100AD400E0932303A1E2B0E00E94772DE093240386
:100AE400A2E2B0E00E94772DE0932503A3E2B0E0F8
:100AF4000E94772DE0932603A4E2B0E00E94772DB4
:100B0400E0932703A5E2B0E00E94772DE093280349
:100B1400ADE3B0E00E94732D0E94AF22A6E2B0E0E4
:100B24000E94772DE0930F03A7E2B0E00E94772D97
:100B34000E94BE2D36F8AAE2B0E00E94772DE09321
:100B4400110336FE0BC0A8E2B0E00E94772DCE2E32
:100B5400A9E2B0E00E94772DE0930003A091020384
:100B6400A43128F4E0910203EF5FE0930203A09123
:100B74000203A431A1F4E0E0E0932E03E0932F03F9
:100B8400EBE0F0E0E0935503F0935603E8EBE093D9
:100B94003003E0E0E093F403EAE0E0930203A09181
:100BA400F403AB30C1F4E091DE03E0932E03E09153
:100BB400DF03E0932F03E091E003F0E0E0935503BB
:100BC400F0935603E091E103E0933003E0E0E09317
:100BD400F403E0930203A091F403AC30C0F0E0E02E
:100BE400E093DB03E093DC03E093DD03E093DE03B7
:100BF400E093DF030E94BE23E0E0E093E203E0938E
:100C0400E303E093E403E093E503E093F403E8EC07
:100C14005E1630F45394E4E1E51511F4E1E04E2E50
:100C24000E94F623A6E00E94FE23EF83F887E7E202
:100C3400E0937A000E94F623A0E00E9405243B97EB
:100C4400C8F1A0E00E94FE23662777270E940A24A9
:100C5400A8EEB3E080E090E00E94BD2CDF01CB0160
:100C64000E941324662777270E94FF2C0E940A24DF
:100C7400AFE8B3E00E94AE2A0E944E2DE091080333
:100C8400EF5FE0930803E0910703A0910803AE1718
:100C940078F00E941824E0938703F093880360930C
:100CA400890370938A0323FC03C0E0E0E093080304
:100CB400E894F3F80E9421240E9492230E9428249D
:100CC400A2E00E94FE23DF01E5E0F0E00E94C22CD6
:100CD4008E2E0E9421240E94AC238AE48A95F1F787
:100CE4000E949F230E942824A7E00E9405240E94BA
:100CF4002F240E942124E7EAE0937A00A5E00E94D1
:100D040005241E2F0E942124E7EAE0937A00A0E044
:100D14000E940524AE2E0E942124E0911103E030AC
:100D240009F08FC0E1E0E51591F50E943424E2E377
:100D3400F0E00E946C2C0E2E0E9439240E94662C36
:100D4400E02111F0E5E0EA8BA12FE2E30E94552CAB
:100D54000E2EEAEF0E94502CE02111F0E6E0EA8B1F
:100D64000E9439240E946C2C0E2E0E943D24E029FE
:100D740011F0E7E0EA8BA12FEAEF0E94552C0E2E2A
:100D8400EEE10E94502CE02911F0E8E0EA8B0E9489
:100D940039240E946C2C0E94432439F0E1E0EA8B50
:100DA400E8E2F0E00E942F2407C00E943D240E9444
:100DB400432411F0E2E0EA8BA12FEAEF0E94552CC4
:100DC4000E94432411F0E3E008C0A12FEEE10E9449
:100DD400502C0E94432419F0E4E0EA8B1CE30E94A7
:100DE4004F240E943C2C0E9457240E943C2CE0215A
:100DF400E1290E2EAA89E1E00E94372C0E2AE2E0B6
:100E04000E94372CE02929F0E12FF0E00E942F24E2
:100E140018E20E944F240E94372C0E9457240E94FB
:100E2400372CE021E12911F00E946124AA890E9453
:100E34006724AA89E8E00E94372CE02909F018E227
:100E440002C0E0E0EA8B0E946C240E9472240E949B
:100E5400502CE021D1F06894F3F8013021F4F39898
:100E6400F49A02E012C0023059F4F498F59AAE8D67
:100E7400A13010F003E003C0F598F39A01E005C037
:100E8400033019F4F598F39A01E00E943424D397BF
:100E940008F457C00E947C240E948124E02F0E9401
:100EA400882420F0E8ECF0E00E942F24E02F0E9438
:100EB40098240E94A824AC91A13008F441C00E9457
:100EC400AF240E94B8240E94B92D4CF40E94A82497
:100ED4000E94C4240E94F72B0E94CF2423C00E94A6
:100EE400D8240E94DA24EF930E94D8240E94E32499
:100EF400AF91EA2379F00E94A8240E94C4240E949E
:100F0400FC2BA0937703B093780380937903909399
:100F14007A0308C00E94D8240E94EC241CF00E948A
:100F2400F6240EC0A0917703B091780380917903E1
:100F340090917A030E9405250E94FF2C0E942F2481
:100F440004C00E9461240E94F6240E940A250E9483
:100F540010250E220E941525E02139F0E091350379
:100F6400E0931F036894F0F821F80E947C243097E2
:100F740021F4E0E0E093200306C0A0912003A23016
:100F840010F4E89425F80E947C24E0933903F0934C
:100F94003A030E947C24309719F4E89421F813C092
:100FA400A0E021FCA1E0E0E00E94372C0E2EA091ED
:100FB4001F030E941C2539F0E0E0E0931F030E9408
:100FC4006124E89422F8E09104030E943424F0E0C0
:100FD400AE17BF0720F0E0913503E0930403E091DE
:100FE4000403F0E035970E943424AE17BF07B0F431
:100FF400E0913503E0930403A0E025FCA1E0E1E0E7
:101004000E94372C0E2E0E94212541F0E2E0E0934D
:101014002D03E89425F8E0E0E0932003A0911F035A
:10102400A13080F0689422F80E947C24A0911F03D0
:10103400B0E0AE17BF0728F0E0911F03F0E00E9474
:101044002F2402C0E89422F80E9429250E942C250E
:101054000E94822C0E22A0912A030E9433251E2E68
:101064000E9429250E942C250E947A2C0E22A091F0
:101074002B030E9433251E2A0E942925A12FE2E377
:101084000E94552CE021E12979F00E946124A0916D
:101094002D03A13021F4EAE0F0E00E942F24E09136
:1010A4002D03E150E0932D030E9438250E22A0E089
:1010B40031FCA1E00E94332531F0689431F80E949C
:1010C4007C240E944E250E943825E02161F10E9473
:1010D40053250E945B25A4F0A0918303B09184035F
:1010E400EB85FC85EA1BFB0BA3E0B0E00E94B82C67
:1010F4000E946325AE1BBF0BA0936503B0936603E8
:101104000E9453250E94AE2D2CF40E94682532972C
:101114000E944E25A0916603AA232AF4E0E0E093FE
:101124006503E09366030E946D250E94B42D74F557
:101134000E946D250E94FC2B0E945B2574F0AB85F8
:10114400BC85E0918303F0918403EA1BFB0B0E94AE
:101154006325EA0FFB1F0E944E250E946D250E9405
:10116400FC2BA230E0E0BE07E0E08E07E0E09E0743
:101174002CF00E94682531960E944E250E9463251A
:10118400A93CE0E0BE0714F00E94C5230E94682534
:101194000E943424AE17BF0710F4E89431F80E947B
:1011A40068250E943424EA17FB0720F40E9468256E
:1011B4000E942F240E947A250E94F12B0E2EA0E07B
:1011C40032FCA1E00E94332541F0689432F80E9479
:1011D4008925E0936703F09368030E947A250E94AF
:1011E400CB2B09F008F435C00E948E25DF01CB011A
:1011F400E0E0F0E060E070E40E94CB2B09F008F43A
:1012040010C00E948E25A0E0B0E080E890E40E9427
:10121400382B0E949D250E94A225A7E6B3E00E94D8
:10122400DE220E948E250E94A42D54F4E8A1F0E051
:101234000E949D25AE1BBF0BA0936703B093680368
:10124400A0916803AA232AF4E0E0E0936703E09303
:1012540068030E947A250E94CB2BC0F50E94A72523
:10126400DF01CB01E0E0F0E060E470E40E94CB2B0E
:1012740009F008F414C00E94A725A0E0B0E080EAB9
:1012840090E40E94382BDF01CB010E94B2250E941A
:10129400B7250E94E82AA7E6B3E00E94DE220E9456
:1012A400A7250E94A42D54F4EF8DF0E00E949D2503
:1012B400EA0FFB1FE0936703F09368030E949D25E8
:1012C400A13DE7E0BE0714F00E94CC230E948925CB
:1012D400DF010E94B225AE17BF0710F4E89432F87C
:1012E4000E948925DF010E94B225EA17FB0720F43A
:1012F4000E949D250E94BC250E94C1250E94822C2B
:101304000E2EA0E034FCA1E00E94332531F0689455
:1013140034F80E9489250E94C8250E94C1250E9494
:10132400B42D5CF50E94CD250E945B259CF0E091D4
:101334001403F0E0A0917F03B0918003AE1BBF0BB8
:10134400E3E0F0E00E94D625AE1BBF0BA0936F0331
:10135400B09370030E94CD250E94AE2D2CF40E9400
:10136400DD2532970E94C825A0917003AA232AF490
:10137400E0E0E0936F03E09370030E94C1250E94B4
:10138400B92D8CF50E94E225A430E0E0BE07E0E030
:101394008E07E0E09E078CF0A0911403BB27E09138
:1013A4007F03F0918003AE1BBF0BE2E0F0E00E94EC
:1013B400D625EA0FFB1F0E94C8250E94E2250E9441
:1013C400AE2D2CF40E94DD2532960E94C825A091F2
:1013D4006F03B0917003A13DE7E0BE0724F0E0ED98
:1013E400F7E00E94C8250E948925DF010E94DD25BF
:1013F400AE17BF0710F4E89434F80E948925DF0182
:101404000E94DD25EA17FB0730F4A0916F03B09129
:1014140070030E94BC251333E0F0E0E0E093060380
:10142400A0911F03A13018F0E2E0E0932D03E0E067
:10143400E0931F03E12FF0E0F2970E94B725A6EF97
:10144400B8E28CE99FE30E94382B0E94752A1E2F74
:1014540001C010E00E947C24E987FA87113010F063
:10146400299A01C02998A82DE4E60E94502C6E2FD9
:101474000E2E0E94F2250E22AE81EDE50E943C2C38
:101484000E94F9251E2E062E0E94F2250E220E948D
:101494001025E0211E2A0E9489230E947F230E9496
:1014A4005A2C0E9400260E948423E021E12931F174
:1014B400E0913D03F0913E03ADE2B0E00E940826C6
:1014C4000E940E260E94B4220E9466230E941B26BC
:1014D4000E942026EC2DA8E2B0E00E942426E09190
:1014E4000003A9E2B0E00E94932D0E948E235F982E
:1014F400A8EEB3E00E94382A5F98FECFAB2D0E947D
:101504002A260E941025E02131F0E894F2F827F809
:10151400E0E0E09334030E942F260E941025E0218E
:1015240071F0E0913403EF5FE0933403A09134034E
:10153400AA3029F4E0E0E0933403E09329030E9405
:101544002F260E943C260E220E941025E02131F114
:101554006894F2F8E0912903EF5FE0932903A091E6
:101564002903E3E00E94432619F0E1E0E093290314
:10157400A0912903E4E00E94432619F0E2E0E093FD
:101584002903A0912903E4E00E94372C0E2EA12FF9
:101594000E941C2519F0E3E0E0932903E09129035C
:1015A400E03031F4E0E0E093B400F7982A981DC0ED
:1015B400A0912903A13031F4E0911A03E093B4001F
:1015C4002A9813C0A0912903A23031F4F79AEFEFBF
:1015D400E093B4002A9809C0A0912903A33029F408
:1015E400F79AEFEFE093B4002A9A0E9434240E9401
:1015F4004E220E2EA12FE0E00E94552C0E220E94B6
:10160400212501F1E0910303EF5FE0930303A0912F
:101614000303E5E00E94552C0E2EE4E10E94502CB9
:10162400E02141F0E0910303E170AFEFEA02F00141
:10163400E093B400A0910303A03118F0E0E0E0933C
:10164400030326C0A0E030FCA1E0E1E00E94372CB7
:101654000E2EA09129030E943325D1F0E09133038B
:10166400EF5FE0933303A0913303A13019F4EFEF5C
:10167400E093B400A0913303A33019F4E0E0E093C5
:10168400B400A0913303A43019F4E0E0E0933303F1
:10169400E0911903E093B300EAE0E91518F4E89443
:1016A400F1F826F80E944826A0E026FCA1E00E945A
:1016B4004E26A0E0F1FCA1E00E944E260E941025D7
:1016C400E02139F16894F1F8E0910E03EF5FE093C3
:1016D4000E03E0E0E98BA989A53088F40E94532623
:1016E400A081A13018F0E5E0E98B05C0E0910E037C
:1016F400EF5FE0930E03E989EF5FE98BECCFA091F4
:101704000E03A53018F0E0E0E0930E030E94532688
:1017140020810E944826A0911C03EFEF0E94502CC8
:10172400E02121F0E0911C03EF5F03C0E894F1F89D
:10173400E0E0E0931C03A0911C03A43109F034C140
:10174400AE81E0E00E944B2C0E2E0E941025E02179
:1017540019F0EE81E150EE83233610F423E624C120
:1017640021E0E0E0E0930E03E0911303A0E0B0E099
:101774000E942426E0911403A1E0B0E00E942426F4
:10178400E0911503A2E0B0E00E942426E091170343
:10179400A3E0B0E00E942426EC8DA4E0B0E00E9417
:1017A4002426ED8DA5E0B0E00E942426EE8DA6E06F
:1017B400B0E00E942426E0911803A7E0B0E00E9464
:1017C4002426E0911903A8E0B0E00E942426E091C9
:1017D4001A03A9E0B0E00E942426E0911D03AAE0C8
:1017E400B0E00E9424260E941324ABE2B0E00E94E1
:1017F4000826E88DA4E1B0E00E942426E98DA5E145
:10180400B0E00E942426EA8DA6E1B0E00E942426DE
:10181400EC89ABE0B0E00E942426ED89ACE0B0E0B6
:101824000E942426EE89ADE0B0E00E942426EB85D8
:10183400FC85AFE2B0E00E940826E0912A03AEE006
:10184400B0E00E942426E0912C03AFE0B0E00E94B7
:101854002426E0912B03A0E1B0E00E942426E32F8C
:10186400A1E1B0E00E942426EF85F889A1E3B0E06D
:101874000E940826E8A1A2E1B0E00E942426EF8D90
:10188400A3E1B0E00E9424260E940E260E9459265D
:10189400A5E3B0E00E940826E0915F03F0916003A5
:1018A400A9E3B0E00E940826E0E023FCE1E0A7E120
:1018B400B0E00E9424260E948923A7E3B0E00E949E
:1018C4000826E0910703A8E1B0E00E942426E091F5
:1018D4000903A9E1B0E00E942426E0910A03AAE1E9
:1018E400B0E00E942426E0910B03ABE1B0E00E943B
:1018F4002426E0910C03ACE1B0E00E942426E091A0
:101904000D03ADE1B0E00E9424260E94B4220E949F
:1019140066230E941B26E0912103AEE1B0E00E9401
:101924002426E0912203AFE1B0E00E942426E09156
:101934002303A0E2B0E00E942426E0912403A1E264
:10194400B0E00E942426E0912503A2E2B0E00E94C8
:101954002426E0912603A3E2B0E00E942426E0912D
:101964002703A4E2B0E00E942426E0912803A5E224
:10197400B0E00E9424260E942026E0910F03A6E2F4
:10198400B0E00E942426E0E036FCE1E0A7E2B0E00B
:101994000E942426E0911103AAE2B0E00E942426CA
:1019A4000E945223E1E04E2E0E944826A0E0F1FC62
:1019B400A1E00E944E26AE81E4E60E94462C0E94DD
:1019C400F92551F06894F1F8EE81EF5FEE83AE8172
:1019D400A43611F4E0E0EE83EAE0E61510F4E894AE
:1019E400F0F80E940A250E9415250E22AE81E0E03F
:1019F4000E94412C0E94F92551F06894F0F8EE8180
:101A0400E150EE83AE81AF3F11F4E3E6EE830E9432
:101A14006C24A22FE3E60E94372CE021C1F00E943F
:101A24005E26A9F4A0913103A43119F4E7E0E09310
:101A34003103E0E0E0933203E894F3F8A09131033A
:101A4400A33028F0E0913103E150E0933103AB2D52
:101A5400EAE00E94502C0E2EA22FE3E60E94372CBF
:101A6400E021C1F00E945E26A9F4A0913103A431C3
:101A740019F4E7E0E0933103E0E0E0933203E89403
:101A8400F2F8A0913103A33028F0E0913103E15042
:101A9400E0933103AB2D0E942A26AA2DEAE00E948E
:101AA400552CE02131F0E0E0E0933203E4E1E093EF
:101AB4003103EAE0EA1510F4E894F3F80E946C2488
:101AC4000E9472240E94372CE02109F499C2689480
:101AD400F3F8AE81A13049F4A0911303A13028F4A6
:101AE400E0911303EF5FE0931303AE81A23049F456
:101AF400A0911403A23328F4E0911403EB5FE09364
:101B04001403AE81A33049F4A0911503A43628F43C
:101B1400E0911503EF5FE0931503AE81A43049F41F
:101B2400A0911703A83228F4E0911703EF5FE09324
:101B34001703AE81A53031F4AC8DA43618F4EC8DC6
:101B4400EF5FEC8FAE81A63031F4AD8DA43618F47E
:101B5400ED8DEF5FED8FAE81A73031F4AE8DA436FD
:101B640018F4EE8DEF5FEE8FAE81A83049F4A091AA
:101B74001803AF3F28F4E0911803EF5FE0931803D4
:101B8400AE81AC3049F4A0910F03A03328F4E09166
:101B94000F03E45FE0930F03AE81AD3069F4A091CD
:101BA4003F03B0914003A433E8E0BE0728F40E9449
:101BB400132431960E94D323AE81AE3031F4A88D24
:101BC400A43618F4E88DEB5FE88FAE81AF3031F4C2
:101BD400A98DA43618F4E98DEB5FE98FAE81A031AD
:101BE40031F4AA8DA43618F4EA8DEB5FEA8FAE8146
:101BF400A13131F4AC89A83C18F4EC89EB5FEC8B8F
:101C0400AE81A23131F4AD89A83C18F4ED89EB5FC3
:101C1400ED8BAE81A33131F4AE89A83C18F4EE8982
:101C2400EB5FEE8BAE81A43169F4A0914F03B091C8
:101C34005003A835E2E0BE0728F40E9489237E966B
:101C44000E94F123AE81A53189F4A0910F03EAE04B
:101C5400EA9FF001EA5BFF4FAB85BC85AE17BF0777
:101C640028F4EB85FC853196EB87FC87AE81A631A1
:101C740049F4A0912A03A13028F4E0912A03EF5FEC
:101C8400E0932A03AE81A73149F4A0912C03A23337
:101C940028F4E0912C03EF5FE0932C03AE81A8318C
:101CA40049F4A0912B03A13028F4E0912B03EF5FBA
:101CB400E0932B03AE81A93191F4A32FEFE00E94AE
:101CC40069260E94332509F03F5FA32FEEE10E94AD
:101CD4006926E1E00E94372CE02109F03F5FAE81E4
:101CE400AA3159F40E947026AC3BE2E0BE0728F406
:101CF4000E94592631960E94E323AE81AB3191F4C0
:101D04000E94C622A73EE3E0BE07E0E08E07E0E0C3
:101D14009E0740F40E948922EF5FFF4F6F4F7F4F71
:101D24000E94E823AE81AC3161F4A0E023FCA1E081
:101D3400A13038F4E0E023FCE1E0EF5F0E94BE2D27
:101D440023F8AE81AD3169F40E944922AE3DE3E04F
:101D5400BE0738F40E942A223A96E0934703F09390
:101D64004803AE81AE3169F40E945322A835E2E003
:101D7400BE0738F40E9436223A96E0935303F09358
:101D84005403AE81AF3149F4A0910703AA3028F47B
:101D9400E0910703EF5FE0930703AE81A03249F4BB
:101DA400A0910903AB3028F4E0910903EF5FE093BD
:101DB4000903AE81A13249F4A0910A03AB3028F49F
:101DC400E0910A03EF5FE0930A03AE81A23249F483
:101DD400A0910B03AB3028F4E0910B03EF5FE09389
:101DE4000B03AE81A33249F4A0910C03AB3028F469
:101DF400E0910C03EF5FE0930C03AE81A43249F44D
:101E0400A0910D03AB3028F4E0910D03EF5FE09354
:101E14000D03AE81A53249F4A0912103A13028F429
:101E2400E0912103EF5FE0932103AE81A63249F4F0
:101E3400A0912203A13028F4E0912203EF5FE09304
:101E44002203AE81A73249F4A0912303A13028F4E0
:101E5400E0912303EF5FE0932303AE81A83249F4BA
:101E6400A0912403A13028F4E0912403EF5FE093D0
:101E74002403AE81A93249F4A0912503A13028F4AA
:101E8400E0912503EF5FE0932503AE81AA3249F484
:101E9400A0912603A33028F4E0912603EF5FE0939A
:101EA4002603AE81AB3249F4A0912703A13028F474
:101EB400E0912703EF5FE0932703AE81AC3249F44E
:101EC400A0912803A13028F4E0912803EF5FE09368
:101ED4002803AE81AD3291F40E945823AF39E6E86D
:101EE400BE07E1E08E07E0E09E0740F40E94402335
:101EF400E65FFF4F6F4F7F4F0E944923AE81AE32A2
:101F040059F40E947526A031E7E2BE0728F40E9426
:101F1400AA223A960E94AF22AE81AF3261F4A0E0C9
:101F240036FCA1E0A13038F4E0E036FCE1E0EF5FFC
:101F34000E94BE2D36F8AE81A03349F4A09111035E
:101F4400A13028F4E0911103EF5FE0931103AE8117
:101F5400AC3549F4A0910603AA3F28F4E0910603A6
:101F6400EB5FE0930603AE81AD3531F4A9A1A73050
:101F740018F4E9A1EF5FE9A3AE81AE3559F4AF855A
:101F8400B889A83BEBE0BE0728F4EF85F8893196C1
:101F9400EF87F88BAE81AF3531F4A8A1AA3018F4DD
:101FA400E8A1EF5FE8A3AE81A03631F4AF8DAA308B
:101FB40018F4EF8DEF5FEF8FAE81A13649F4A09155
:101FC4001D03AC3328F4E0911D03EF5FE0931D0380
:101FD400AE81A23649F4A0911A03AA3F28F4E091F5
:101FE4001A03E65FE0931A03AE81A33649F4A09185
:101FF4001903AA3F28F4E0911903E65FE09319035B
:10200400EAE0EB1510F4E894F2F8AB2DEAE00E9454
:10201400502C0E2E0E943C260E94F92509F47FC202
:102024006894F2F8AE81A13049F4A0911303A13071
:1020340028F0E0911303E150E0931303AE81A23042
:1020440049F4A0911403AB3028F0E0911403E55057
:10205400E0931403AE81A33049F4A0911503AD338A
:1020640028F0E0911503E150E0931503AE81A4300C
:1020740049F4A0911703A53128F0E0911703E1502A
:10208400E0931703AE81A53031F4AC8DA13018F084
:10209400EC8DE150EC8FAE81A63031F4AD8DA130E2
:1020A40018F0ED8DE150ED8FAE81A73031F4AE8D97
:1020B400A13018F0EE8DE150EE8FAE81A83049F4D6
:1020C400A0911803A13028F0E0911803E150E093A7
:1020D4001803AE81AC3049F4A0910F03A93128F064
:1020E400E0910F03EC50E0930F03AE81AD3069F43F
:1020F400A0913F03B0914003AD36E7E0BE0728F05E
:102104000E94132431970E94D323AE81AE3031F460
:10211400A88DA63018F0E88DE550E88FAE81AF3079
:1021240031F4A98DA63018F0E98DE550E98FAE8120
:10213400A03131F4AA8DA63018F0EA8DE550EA8F6B
:10214400AE81A13131F4AC89A13018F0EC89E550AD
:10215400EC8BAE81A23131F4AD89A13018F0ED8958
:10216400E550ED8BAE81A33131F4AE89A13018F086
:10217400EE89E550EE8BAE81A43161F4A0914F035A
:10218400B09150030E94AA2D28F40E9489237E97BF
:102194000E94F123AE81A53189F4A0910F03EAE0F6
:1021A400EA9FF001E654F040AB85BC85EA17FB07D3
:1021B40028F4EB85FC853197EB87FC87AE81A6314B
:1021C40049F4A0912A03A13028F0E0912A03E150B8
:1021D400E0932A03AE81A73149F4A0912C03A230E5
:1021E40028F0E0912C03E150E0932C03AE81A83158
:1021F40049F4A0912B03A13028F0E0912B03E15086
:10220400E0932B03AE81A93119F4323008F0315038
:10221400AE81AA3159F40E947026A935E2E0BE07C6
:1022240028F00E94592631970E94E323AE81AB31F6
:1022340091F40E94C622AB30E0E0BE07E0E08E07D6
:10224400E0E09E0740F00E948922E150F0406040A7
:1022540070400E94E823AE81AC3159F4A0E023FC25
:10226400A1E0A13030F0A0E023FCA1E00E947A2696
:1022740023F8AE81AD3161F40E9449220E94AA2D57
:1022840038F40E942A223197E0934703F0934803DD
:10229400AE81AE3161F40E9453220E94AA2D38F41B
:1022A4000E9436223197E0935303F0935403AE8196
:1022B400AF3149F4A0910703A23028F0E09107035D
:1022C400E150E0930703AE81A03249F4A0910903E1
:1022D400A23028F0E0910903E150E0930903AE81B4
:1022E400A13249F4A0910A03A13028F0E0910A0335
:1022F400E150E0930A03AE81A23249F4A0910B03AA
:10230400A13028F0E0910B03E150E0930B03AE8180
:10231400A33249F4A0910C03A13028F0E0910C03FE
:10232400E150E0930C03AE81A43249F4A0910D0373
:10233400A13028F0E0910D03E150E0930D03AE814C
:10234400A53249F4A0912103A13028F0E0912103A2
:10235400E150E0932103AE81A63249F4A091220317
:10236400A13028F0E0912203E150E0932203AE81F2
:10237400A73249F4A0912303A13028F0E09123036C
:10238400E150E0932303AE81A83249F4A0912403E1
:10239400A13028F0E0912403E150E0932403AE81BE
:1023A400A93249F4A0912503A13028F0E091250336
:1023B400E150E0932503AE81AA3249F4A0912603AB
:1023C400A13028F0E0912603E150E0932603AE818A
:1023D400AB3249F4A0912703A13028F0E091270300
:1023E400E150E0932703AE81AC3249F4A091280375
:1023F400A13028F0E0912803E150E0932803AE8156
:10240400AD3269F40E9458230E94AE2D40F40E941C
:102414004023E150F040604070400E944923AE8167
:10242400AE3251F40E9475260E94AA2D28F40E940F
:10243400AA2231970E94AF22AE81AF3259F4A0E0B4
:1024440036FCA1E0A13030F0A0E036FCA1E00E940F
:102454007A2636F8AE81A03349F4A0911103A13055
:1024640028F0E0911103E150E0931103AE81AC3503
:1024740049F4A0910603A13028F0E0910603E55049
:10248400E0930603AE81AD3531F4A9A1A13018F073
:10249400E9A1E150E9A3AE81AE3559F4AF85B8891D
:1024A400A13DE7E0BE0728F0EF85F8893197EF8773
:1024B400F88BAE81AF3531F4A8A1A13018F0E8A1B2
:1024C400E150E8A3AE81A03631F4AF8DA13018F00D
:1024D400EF8DE150EF8FAE81A13649F4A0911D0339
:1024E400A13028F0E0911D03E150E0931D03AE817B
:1024F400A23649F4A0911A03AB3028F0E0911A03F4
:10250400EA50E0931A03AE81A33649F4A09119036B
:10251400A13028F0E0911903EA50E093190323FC59
:1025240028C0E0912F03A7ECB3E0FF2766277727A5
:102534000E94AE2A0E944E2D0E9481260E94AE2D3A
:102544003CF40E948A260E9493260E949A2609C07F
:10255400E0E0E093B703E093B803E093B903E093BA
:10256400BA030E948A26A1E7B3E00E94DE220E94F9
:10257400A32623FE52C0EF81F8850E94B7250E944E
:10258400582D0E94532DE0E0F0E060E874E40E94CE
:10259400862BA0E0B0E48CE995E40E94382BDF019F
:1025A400CB01EF85F889662777270E94AE2A0E941F
:1025B400A522DF01CB01E3E3F3E365E872E40E94C3
:1025C400862BE093C703F093C8036093C903709309
:1025D400CA03A0911003A13048F4E0E0E093C703DC
:1025E400E093C803E093C903E093CA030E948A26D8
:1025F4000E949A26E0910703A0910803AE1768F0A1
:102604000E9481260E946623A1E7B3E00E94DE2295
:102614000E94A326E0E0E0930803F0915503E0E074
:10262400DF01E0913003F0E0EA0FFB1FA7E9B3E01C
:102634000E942F220E94A726A0E0B0E080E192E44D
:102644000E94862B7F936F93FF93EF930E947026D3
:102654000E94B026AF91BF918F919F9166277727F3
:102664000E94AE2A0E94382BE0939703F0939803BC
:102674006093990370939A030E94B526E0E0F0E01A
:1026840060E87FE30E94F12B0E2E0E94B526E0E065
:10269400F0E068EC72E40E94EB2BE021E9F00E9488
:1026A400A7260E949326AFE7B3E00E94772A0E94F0
:1026B4004E2D0E94A726E0939B03F0939C03609306
:1026C4009D0370939E030E94B5260E94DF23A1E41C
:1026D400B3E00E94612215C0E0E0E0937F03E09341
:1026E4008003E0938103E0938203E0939B03E093F0
:1026F4009C03E0939D03E0939E03E0934103E093E6
:1027040042030E94EA220E9461230E94F12BEF936C
:102714000E94BE260E94F12BAF91EA23C1F10E94D0
:102724007722E0E0F0E068EC72E40E94862B0E94DD
:10273400C6220E945D2D0E94A5220E94C026A0915F
:102744009303B09194038091950390919603E0E0F4
:10275400F0E064E172E40E94382BDF01CB010E94B7
:1027640001230E94862BA0E0B0E080E291E40E9465
:10277400382B0E94C026E0919303F091940360915A
:10278400950370919603DE0114960E94DE220E9446
:102794000A25A0911B03EDEF0E94502C0E220E94EB
:1027A4001025E02129F0E0911B03EF5FE0931B0368
:1027B400A62D0E942A26A0911B03EFEF0E94502C05
:1027C4000E220E941025E02129F0E894F0F8E0E0C0
:1027D400E0931B03A0911B03EEE10E94372C0E2E05
:1027E4000E941025E02119F0E1E0E0931E03E0913E
:1027F4001D03E03019F4E0E0E0931E030E946F2310
:102804000E9461230E94822C0E940026A0911E0334
:102814000E941C2519F0E1E0E0931E03A0911E0321
:10282400AC3309F41FEFA0910603A13028F0E09126
:102834000603F0E00E942F244420C9F4E02FF0E0C6
:1028440034960E943424AE0FBF1FE12F0E94C92684
:10285400A4E00E940B22A02F0E94D326A09135034E
:102864000E940B22A12F0E940B220E94D826E1E095
:10287400E41509F057C04424A09115030E94E126F1
:10288400E0931603F0E0BC96DF01E0911203F0E060
:10289400AE0FBF1FE0911303F0E0AE0FBF1FE09136
:1028A4001403F0E0AE0FBF1FE0911703F0E0AE0F8A
:1028B400BF1FEC8DF0E0AE0FBF1FED8DF0E0AE0F4B
:1028C400BF1FEE8DF0E0AE0FBF1FE09118030E9412
:1028D400C926ACE20E940B22A09112030E940B2293
:1028E400A09113030E940B22A09114030E940B22B7
:1028F400A09116030E940B22A09117030E940B22A1
:10290400AC8D0E940B22AD8D0E940B22AE8D0E94D5
:102914000B22A09118030E94D326A0E00E94D32684
:102924000E94D826233608F06EC50E9453262081C3
:10293400A0E0F799A1E0EA2FE295E07F0E2EA0E057
:10294400F399A1E0EA2FEE0FEE0F0E0EA0E0F4993A
:10295400A1E0EA2FEE0FA02DAE0FE0E0F599E1E043
:10296400EA0FEAA3EAE0EFABE8AFE9AFEAAFEBAF17
:10297400ECAFEDAF0E94E726EAE00E94EF26EAE022
:102984000E94F426EAE00E94F926EAE00E94FE266C
:10299400EAE0DE01AB5BBF4FEC93E89435F8E091DD
:1029A4002603E03021F40E940327E00DEBA3A0915D
:1029B4002603A13081F4A0E022FCA1E0EA2FEE0F6F
:1029C400E75F0E2EA0E022FCA1E0EA2FEE0FEE0F4F
:1029D400E00D0E941C27A0912603A23099F40E94C6
:1029E40003270E0EA0E022FCA1E0EA2F0E94362766
:1029F4000E0EA0E022FCA1E0EA2FE295E07FEE0FAC
:102A0400E00DEBA3A0912603A33031F4E0E022FC17
:102A1400E1E0E85F0E941C27A0910F03A83109F0B0
:102A240041C00E943B27A23DE0E0BE07E0E08E07E4
:102A3400E0E09E071CF0E1E0E09301030E944927D7
:102A4400A83FE0E0BE07E0E08E07E0E09E071CF050
:102A5400E3E0E09301030E944927AF3FE0E0BE07B3
:102A6400E0E08E07E0E09E071CF0E7E0E09301035E
:102A74000E944927A430E1E0BE07E0E08E07E0E0D1
:102A84009E071CF0EFE0E09301030E944927AE305B
:102A9400E1E0BE07E0E08E07E0E09E071CF0EFE116
:102AA400E0930103A0910F03A43209F041C00E94F6
:102AB4003B27A633E1E0BE07E0E08E07E0E09E0797
:102AC4001CF0E1E0E09301030E944927AA34E1E00D
:102AD400BE07E0E08E07E0E09E071CF0E3E0E09331
:102AE40001030E944927AE35E1E0BE07E0E08E070E
:102AF400E0E09E071CF0E7E0E09301030E94492711
:102B0400A836E1E0BE07E0E08E07E0E09E071CF097
:102B1400EFE0E09301030E944927AC37E1E0BE07F0
:102B2400E0E08E07E0E09E071CF0EFE1E093010394
:102B3400A0910F03A03309F041C00E943B27A6389F
:102B4400E1E0BE07E0E08E07E0E09E071CF0E1E074
:102B5400E09301030E944927AC3CE1E0BE07E0E0BA
:102B64008E07E0E09E071CF0E3E0E09301030E947F
:102B74004927A63DE1E0BE07E0E08E07E0E09E07BE
:102B84001CF0E7E0E09301030E944927A03EE1E046
:102B9400BE07E0E08E07E0E09E071CF0EFE0E09364
:102BA40001030E944927AF3EE1E0BE07E0E08E0743
:102BB400E0E09E071CF0EFE1E09301030E946F2325
:102BC4000E9452272CF00E945A270E946027E9AFE6
:102BD4000E945A270E94192DEAAFA0917203AA23DA
:102BE4007AF4E0E4EFABA0917103B0917203AD39D4
:102BF400EFEFBE0714F4689435F80E946B2702C007
:102C0400E89435F80E947B271A972CF00E948027BD
:102C14000E948427EFAB0E9480270E94072DE8AF13
:102C24000E9449270E948C270E946027EBAF0E94D4
:102C340091270E946027ECAF0E9491270E94192DD2
:102C4400EDAF0E944927A639E0E0BE07E0E08E0719
:102C5400E0E09E073CF4E0E4EBAFECAFEDAFE0E086
:102C6400E0930103213009F04CC00E9497270E9491
:102C7400A127A83EE3E0BE0788F0ECA1E05EECA348
:102C84000E94A6270E94AB270E94B7270E94BC2758
:102C94000E94C8270E94B026DF0115C0ECA1E056AF
:102CA400ECA30E94A127A436E0E0BE0720F00E9416
:102CB400A6270E94BC270E94B7270E94B0260E9424
:102CC400CD270E94C827EAE0F0E00E94D527A09112
:102CD4000003AA3010F0E2E0EEAFA09100030E94DE
:102CE400DA27EFAF0E94E027AC2DB0E00E94E52781
:102CF4000E94E8273B96BF01AC2D0E94DA27DB0136
:102D0400EC93223009F075C0ECA1E05CECA30E94C6
:102D14005823A03AE6E8BE07E1E08E07E0E09E070C
:102D240080F0FE01F6963A96FF93EF930E945823A3
:102D3400E0EAF6E861E070E00E94ED27AF91BF9110
:102D4400EC930E9458230E94F82780F0FE01F69627
:102D54003B96FF93EF930E945823E0E1F7E260E093
:102D640070E00E94ED27AF91BF91EC930E9458232D
:102D74000E94002870F0FE01F6963C96FF93EF93B4
:102D84000E9458230E9405250E94ED27AF91BF9110
:102D9400EC930E9458230E94082870F0FE01F696D6
:102DA4003D96FF93EF930E9458230E948C270E9424
:102DB400ED27AF91BF91EC930E9458230E945227B4
:102DC40060F0FE01F6963E96FF93EF930E94102862
:102DD4000E94ED27AF91BF91EC93FE01F6963F96CA
:102DE400FF93EF930E9410280E94152DAF91BF917D
:102DF400EC93233009F096C0E7E70E941628A091CF
:102E04008E03AA2392F4E0918B03F0918C036091DA
:102E14008D0370918E030E94052CE0938B03F09335
:102E24008C0360938D0370938E030E94BE260E94D0
:102E3400A52277231AF4E0E40E94FE260E94BE260F
:102E44000E94A5220E941D2818F4E0E40E94F9269D
:102E54000E94BE260E94A5220E94262818F4E0E4BF
:102E64000E94F4260E94BE260E94A5220E942F28BA
:102E740018F4E0E40E94EF260E9432280E94F8270A
:102E840084F0FE01F6963B96FF93EF930E9432285E
:102E9400E0E1F7E260E070E00E946027AF91BF914B
:102EA400EC930E9432280E94002874F0FE01F696EA
:102EB4003C96FF93EF930E9432280E9405250E94BE
:102EC4006027AF91BF91EC930E9432280E9408289A
:102ED40064F0FE01F6963D96FF93EF930E9432282C
:102EE4000E943B28AF91BF91EC930E9432280E942C
:102EF400522764F0FE01F6963E96FF93EF930E94EC
:102F04003D280E946027AF91BF91EC93FE01F69695
:102F14003F96FF93EF930E943D280E94192DAF9195
:102F2400BF91EC93243009F059C00E944328A0912A
:102F34006E03AA2312F40E9448280E945328772380
:102F44001AF4E0E40E94FE260E9453280E941D28E1
:102F540018F4E0E40E94F9260E9453280E942628CF
:102F640018F4E0E40E94F4260E9453280E942F28BB
:102F740018F4E0E40E94EF260E945928A031E7E209
:102F8400BE0734F00E945E280E946328DB01EC93A4
:102F94000E945928A83EE3E0BE0734F00E94672847
:102FA4000E946C28DB01EC930E945928A436E0E0CF
:102FB400BE0734F00E9470280E947528DB01EC9350
:102FC4000E9459281A9744F00E9479280E9459288F
:102FD4000E94E527DB01EC930E947E28253071F5E1
:102FE4000E944328E0E50E94EF26A091BE03AA2395
:102FF4001AF4E0E40E94F9260E94EA22E0E0F0E0FC
:1030040066EC72EC0E94CB2B18F4E0E40E94F426E8
:103014000E948A28A436E0E0BE0734F00E9470289B
:103024000E948F28DB01EC930E9479280E948A2851
:103034000E94E5270E94E8270E9493282630D9F5AC
:10304400ECA1E058ECA3E0E0EFAFE5E00E949D289E
:10305400E8E70E94EF26AC81BD81A83EE3E0BE070D
:1030640054F00E946728AC81BD81E8EEF3E00E9431
:103074008427DB01EC93AC81BD81A436E0E0BE077C
:1030840054F00E947028AC81BD81E4E6F0E00E9417
:103094008427DB01EC930E947928AC81BD810E94D6
:1030A400E5270E94E8273F96BF01AC81BD810E94BD
:1030B400A228DB01EC93273009F051C0113058F1FC
:1030C400ECE0EFAFA12F0E94E126E436A0E0FA077E
:1030D40054F00E94E027A12FB0E0E8ECF0E00E9459
:1030E4008427DB01EC93A12F0E94E1263A9754F048
:1030F4000E945E28A12FB0E0E4E1F0E00E94842762
:10310400DB01EC930E946728A12F0E94E126DF01D6
:103114000E94A22822C0EBE0EFAF0E94A728E43669
:10312400A0E0FA0740F00E94E027A985BA85E8EC00
:10313400F0E00E94AC280E94A7283A9740F00E9431
:103144005E28A985BA85E4E1F0E00E94AC280E94DB
:1031540067280E94A7280E94AF28DB01EC9328303F
:1031640009F079C00E949727A0916903B0916A037E
:10317400A135EBEFBE0734F4E1E5FBEFE09369031F
:10318400F0936A03A0916903B0916A03A03BE4E061
:10319400BE0734F0EFEAF4E0E0936903F0936A03C6
:1031A400A0916A03AA2352F4E0E40E94F426E09179
:1031B4006903F0916A030E94012C04C0E091690341
:1031C400F0916A03E0936B03F0936C03A0916B039B
:1031D400B0916C03ECE3F0E00E94D52CE09349033A
:1031E400F0934A030E94B528ECE30E94B22CA0910C
:1031F4006B03B0916C03AE1BBF0BA0934B03B09356
:103204004C0324FE1DC00E94B5281A9710F0E2E07A
:10321400EEAF0E94B5280E94BA28EFAF0E94E027C3
:10322400A0914B03B0914C030E94B0260E94CD277D
:103234000E945E28A0914B03B0914C030E94BF28CA
:10324400E3E70E94F926E8E30E94FE26E4E5DE01B6
:10325400AB5BBF4FEC93293009F059C00E94C228E0
:10326400A0916E03AA2312F40E9448280E945328B6
:1032740077231AF4E0E40E94FE260E9453280E9459
:103284001D2818F4E0E40E94F9260E9453280E94A5
:10329400262818F4E0E40E94F4260E9453280E9491
:1032A4002F2818F4E0E40E94EF260E945928A03148
:1032B400E7E2BE0734F00E945E280E946328DB0127
:1032C400EC930E945928A83EE3E0BE0734F00E9424
:1032D40067280E946C28DB01EC930E945928A436CD
:1032E400E0E0BE0734F00E9470280E947528DB01DC
:1032F400EC930E9459281A9744F00E9479280E945E
:1033040059280E94E527DB01EC930E947E282A308D
:10331400D9F40E94C228E0E50E94EF260E948A2880
:10332400A436E0E0BE0734F00E9470280E948F2883
:10333400DB01EC930E9479280E948A280E94E527E9
:103344000E94E8270E9493282B3069F5ECA1E054F1
:10335400ECA30E94C9280E947526A83EE3E0BE079C
:1033640030F00E9467280E9475260E94AB270E94B5
:103374007526A436E0E0BE0730F00E9470280E9453
:1033840075260E94BC270E9479280E9475260E94F7
:10339400B0260E94CD27FE01F6963F96BF010E94FB
:1033A40075260E94BF28AA89A13030F1ECA1EF77DD
:1033B400ECA3E0912E03E170EE0FABA1EA23EBA3A3
:1033C400E058EBA30E94E726E9E70E94EF26E0E538
:1033D4000E94F426E0E50E94F9260E947928AA8931
:1033E400B0E00E94E5270E94E8273F96BF01AA8922
:1033F4000E94DA27DB01EC93F29B05C0EBA1EB7F83
:10340400EBA3EF5FEBA3233609F0CAC451E05031BC
:1034140040F40E94CD28EAE0EC93E89435F85F5F2D
:10342400F6CFAE81EBE50E94D428EAE50E94372C62
:10343400E02911F0E0E3EE83AE81A13311F4ECE571
:10344400EE83EE81E03029F4E0911203F0E0ED87A1
:10345400FE87AE81A13029F4E0911303F0E0ED87FB
:10346400FE87AE81A23029F4E0911403F0E0ED87E9
:10347400FE87AE81A33029F4E0911503F0E0ED87D7
:10348400FE87AE81A43029F4E0911703F0E0ED87C4
:10349400FE87AE81A53021F4EC8DF0E0ED87FE8748
:1034A400AE81A63021F4ED8DF0E0ED87FE87AE818C
:1034B400A73021F4EE8DF0E0ED87FE87AE81A830D1
:1034C40029F4E0911803F0E0ED87FE87AE81A9307E
:1034D40019F4E0E0ED87EE87AE81AA3019F4E0E05C
:1034E400ED87EE87AE81AB3019F4E0E0ED87EE872F
:1034F400AE81AC3029F4E0910F03F0E0ED87FE8754
:10350400AE81AD3021F40E941324ED87FE87AE8195
:10351400AE3021F4E88DF0E0ED87FE87AE81AF3068
:1035240021F4E98DF0E0ED87FE87AE81A03121F42E
:10353400EA8DF0E0ED87FE87AE81A13121F4EC89BC
:10354400F0E0ED87FE87AE81A23121F4ED89F0E051
:10355400ED87FE87AE81A33121F4EE89F0E0ED879B
:10356400FE87AE81A43121F40E948923ED87FE8772
:10357400AE81A53121F4EB85FC85ED87FE87AE8114
:10358400A63129F4E0912A03F0E0ED87FE87AE81AD
:10359400A73129F4E0912C03F0E0ED87FE87AE819A
:1035A400A83129F4E0912B03F0E0ED87FE87AE818A
:1035B400A93121F4E32FF0E0ED87FE87AE81AA3133
:1035C40021F40E945926ED87FE87AE81AB3131F498
:1035D400E0915F03F0916003ED87FE87AE81AC312B
:1035E40031F4E0E023FCE1E0F0E0ED87FE87AE811A
:1035F400AD3121F40E942A22ED87FE87AE81AE31DF
:1036040021F40E943622ED87FE87AE81AF3129F482
:10361400E0910703F0E0ED87FE87AE81A03229F444
:10362400E0910903F0E0ED87FE87AE81A13229F431
:10363400E0910A03F0E0ED87FE87AE81A23229F41F
:10364400E0910B03F0E0ED87FE87AE81A33229F40D
:10365400E0910C03F0E0ED87FE87AE81A43229F4FB
:10366400E0910D03F0E0ED87FE87AE81A53229F4E9
:10367400E0912103F0E0ED87FE87AE81A63229F4C4
:10368400E0912203F0E0ED87FE87AE81A73229F4B2
:10369400E0912303F0E0ED87FE87AE81A83229F4A0
:1036A400E0912403F0E0ED87FE87AE81A93229F48E
:1036B400E0912503F0E0ED87FE87AE81AA3229F47C
:1036C400E0912603F0E0ED87FE87AE81AB3229F46A
:1036D400E0912703F0E0ED87FE87AE81AC3229F458
:1036E400E0912803F0E0ED87FE87AE81AD3231F43E
:1036F400E0915B03F0915C03ED87FE87AE81AE320F
:1037040021F40E94AA22ED87FE87AE81AF3231F404
:10371400E0E036FCE1E0F0E0ED87FE87AE81A03327
:1037240029F4E0911103F0E0ED87FE87AE81AC351A
:1037340029F4E0910603F0E0ED87FE87AE81AD3514
:1037440021F4E9A1F0E0ED87FE87AE81AE3521F4E6
:10375400EF85F889ED87FE87AE81AF3521F4E8A1C6
:10376400F0E0ED87FE87AE81A03621F4EF8DF0E026
:10377400ED87FE87AE81A13629F4E0911D03F0E0C8
:10378400ED87FE87AE81A23629F4E0911A03F0E0BA
:10379400ED87FE87AE81A33629F4E0911903F0E0AA
:1037A400ED87FE87AE81E0E00E94D428E3E00E942A
:1037B400D928E1E10E94D928E2E10E94D928E3E175
:1037C4000E94D928E5E10E94D928EBE10E94D9287A
:1037D400EDE10E94D928EEE20E94372CE02911F095
:1037E400F69A01C0F698A0E0F699A1E0EA2FE795D1
:1037F400E0E0E795ECA3E0E0EBA3EAA3E0930103A8
:10380400AE81B0E0A7FDBFEF0E94E527E9AFAE812E
:10381400B0E0A7FDBFEF0E94A228EAAFAD85BE8548
:10382400A031E7E2BE0740F00E945E28AD85BE8568
:10383400E0E1F7E20E94AC28AD85BE85A83EE3E056
:10384400BE0730F00E946728AD85BE850E94AB2775
:10385400AD85BE85A436E0E0BE0730F00E94702836
:10386400AD85BE850E94BC27AD85BE851A9730F014
:103874000E9479280E94DE280E94CD27FE01F69638
:103884003F96BF01AD85BE850E94BF28EE81E03022
:1038940079F4EDE6EBAFE9E7ECAFE8E7EDAFEDE6A1
:1038A4000E949D28E4E50E94EF26E0E50E94F426AC
:1038B400AE81E1E10E94D428E2E10E94D928E3E14B
:1038C4000E94D928E5E10E94D928EDE10E94D92877
:1038D400EEE20E94372CE02931F00E9479280E9400
:1038E400DE280E94CD27E7EAE0937A00A7E00E9451
:1038F40005240E942F24E7E2E0937A000E94E12845
:10390400EEE00E94D928E1E10E94372CE02911F071
:10391400E1E07E2EAE810E946724AE81EFE00E943A
:10392400D928E2E10E94372CE02911F0E2E07E2E52
:10393400AE81E7E00E94D428E0E10E94D9280E94E9
:10394400E42811F0E3E07E2E0E943424D39708F497
:1039540057C00E947C240E948124E72D0E94882461
:1039640020F0E8ECF0E00E942F24E72D0E94982438
:103974000E94E928AC91A13008F441C00E94F028CB
:103984000E94B8240E94B92D4CF40E94E9280E9498
:10399400F9280E94F72B0E94042923C00E940D29B4
:1039A4000E94DA24EF930E940D290E94E324AF9130
:1039B400EA2379F00E94E9280E94F9280E94FC2B4E
:1039C400A0937B03B0937C0380937D0390937E0349
:1039D40008C00E940D290E94EC241CF00E940F29AB
:1039E4000EC0A0917B03B0917C0380917D039091E4
:1039F4007E030E9405250E94FF2C0E942F2404C0F0
:103A04000E9461240E940F29AE81AD3051F40E94BE
:103A140017290E943B280E9420290E942729E0E2BE
:103A2400EAA3AE81A53151F40E9417290E943B28D4
:103A34000E9420290E942729E0E6EAA30E94E128A7
:103A4400EEE00E94D928E1E10E94372CE029A9F098
:103A54000E943129E4E00E94352918F00E943B2994
:103A6400EBAF0E9434241A9728F00E9441290E9447
:103A7400AF28ECAF0E944329EDAFAE810E946724CA
:103A8400AE81EFE00E94D928E2E10E94372CE029C0
:103A9400A9F00E943129E2E00E94352918F00E9421
:103AA4003B29EBAF0E9434241A9728F00E94412945
:103AB4000E94AF28ECAF0E944329EDAFAE81E7E04E
:103AC4000E94D428E0E10E94D9280E94E428A9F0A9
:103AD4000E943129E1E00E94352918F00E943B2917
:103AE400EBAF0E9434241A9728F00E9441290E94C7
:103AF400AF28ECAF0E944329EDAFAE81A43189F425
:103B04000E9445290E944A29EBAF0E9445290E9440
:103B1400B0260E94AF28ECAF0E9445290E94BA2823
:103B2400EDAFAE81A63129F40E944F29EBE00E944B
:103B3400F426AE81A73129F40E944F29E0E40E94C3
:103B4400F426AE81A83129F40E944F29ECE00E94AA
:103B5400F426AE81A93191F4A091CA03AA2312F4E8
:103B64000E946B270E9480270E948427EBAF0E944B
:103B740080270E94072DECAFE7E7EDAFAE81AA31B5
:103B840089F40E9455290E944A29EBAF0E945529C5
:103B94000E94B0260E94AF28ECAF0E9455290E94D3
:103BA400BA28EDAFAE81AB3171F4ECE7EFAFE7E7E4
:103BB4000E949D28E8E70E94EF260E9479280E942F
:103BC400DE280E94CD27AE81EDE10E94D428EEE1EB
:103BD4000E94372CE029F9F0E3E7EFAFE8E30E9415
:103BE4009D28AE81AD3111F4EEE501C0E8E7DE01B8
:103BF400AF5BBF4FEC930E945A291A9738F00E948A
:103C04005A290E94B0260E94AF28ECAF0E945A297C
:103C14000E94BA28EDAF0E94E128E6E00E94D9286C
:103C2400E7E00E94372CE02911F0E3E7EFAFAE8123
:103C3400EEE00E94D428EFE00E94D928E0E10E943F
:103C4400372CE02941F0EDE6EFAFE9E70E949D282B
:103C5400E4E50E94EF26AE81E1E10E94D428E2E18E
:103C64000E94D9280E94E42819F0E8E70E949D28C0
:103C7400AE81EFE10E944B2C0E2EE5E20E94462C11
:103C8400E02139F0EDE6EBAFE8E5ECAFEE81EF5182
:103C9400EDAFAE81AD3219F4ECA1E05CECA3AE81E2
:103CA400AE3211F40E94C928AE81AD35A9F5E7E71B
:103CB4000E94F426EEE50E94F926E9E30E94FE261E
:103CC400FE01F6963F96A9A1A083E7EAE0937A0065
:103CD4000E94FE23E0933703F0933803E7E2E09376
:103CE4007A000E945F29A436E0E0BE0728F00E9413
:103CF4005F290E944A29EBAF0E945F291A9738F086
:103D04000E945F290E94B0260E94AF28ECAF0E9457
:103D14005F290E94BA28EDAFAE81AE3561F50E94ED
:103D240081260E946623A3E7B3E00E94DE22A091CD
:103D3400CA03AA2352F4E0917303F09174030E941E
:103D4400012CE0937303F09374030E947B27E4E651
:103D5400F0E00E948427EBAF0E9480270E94842712
:103D6400ECAF0E9480270E94072DEDAFEEE5EFAF88
:103D7400E1E00E949D28AE81AF3529F4EEE5EFAF76
:103D8400E2E00E949D28AE81A03629F4EEE5EFAF73
:103D9400E3E00E949D28AE81A23611F4E0E1EAA39B
:103DA40051E0503108F077C00E94CD28EC91E0300A
:103DB40021F40E94CD28EFE3EC930E94CD28AC912E
:103DC400A63021F40E94CD28EDE7EC930E94CD2883
:103DD400AC91A13021F40E94CD28E6E0EC930E943E
:103DE400CD28AC91A23021F40E94CD28EBE5EC93D0
:103DF4000E94CD28AC91A33021F40E94CD28EFE499
:103E0400EC930E94CD28AC91A43021F40E94CD28DB
:103E1400E6E6EC930E94CD28AC91A53021F40E94F3
:103E2400CD28EDE6EC930E94CD28AC91A73021F487
:103E34000E94CD28E7E0EC930E94CD28AC91A830F5
:103E440021F40E94CD28EFE7EC930E94CD28AC9199
:103E5400A93021F40E94CD28EFE6EC930E94CD28EE
:103E6400AC91AA3021F40E94CD28E0E0EC930E94AA
:103E7400CD28AC91AB3021F40E94CD28E1E0EC9345
:103E84000E94CD28AC91AC3021F40E94CD28E8E00A
:103E9400EC935F5F86CFE0910103E695E6950E947F
:103EA4006429EBAD0E946A29EBAD0E947229EBAD47
:103EB4000E947D29EBAD0E948429EBAD0E948B29E1
:103EC400EBAD0E949229EBAD0E949929EEA3E091FB
:103ED4000103E695E695E6950E946429ECAD0E94FF
:103EE4006A29ECAD0E947229ECAD0E947D29EDADEA
:103EF4000E948429EDAD0E948B29EDAD0E94922988
:103F0400EDAD0E949929EFA3E0910103E6950E948B
:103F14006429EDAD0E946A29EDAD0E947229EDADD0
:103F24000E947D29ECAD0E948429ECAD0E948B296E
:103F3400ECAD0E949229ECAD0E949929E8A7EEAD60
:103F44000E946429EFAD0E946A29EFAD0E94722994
:103F5400EFAD0E947D29ECA10E948429ECA10E946E
:103F64008B29ECA10E949229E0910103E170EA2BD4
:103F7400E9A70E949F290E9464290E949F290E9408
:103F8400A4290E949F290E94AA290E949F290E9475
:103F9400B3290E94BD290E949F290E94C1290E9421
:103FA4009F290E94CA290E949F29E295E170EA2B69
:103FB400EAA70E94D3290E9464290E94D3290E945F
:103FC400A4290E94D3290E94AA290E94D3290E94CD
:103FD400B329E2950E9484290E94D8290E94C1290C
:103FE4000E94D8290E94CA290E94D829E295E1702A
:103FF400EA2BEBA7ECA10E94DD290E94D3290E94A1
:104004006A290E94D3290E9472290E94D3290E94FE
:104014007D290E94E1290E9484290E94E1290E94AD
:104024008B290E94E1290E9492290E94E1290E9481
:104034009929ECA70E94D8290E9464290E94D829B2
:104044000E94A4290E94D8290E94AA290E94D82942
:104054000E94B3290E94E6290E9484290E94E12932
:104064000E94C1290E94E1290E94CA290E94E129D3
:10407400E295E170EA2BEDA70E94EB290E946429E6
:104084000E94EB290E94A4290E94EB290E94AA29DC
:104094000E94EB290E94B329EE1FE0E0EE1F0E946C
:1040A40084290E94F0290E94C1290E94F0290E94BB
:1040B400CA290E94F029E295E170EA2BEEA7EBA150
:1040C400E2950E9464290E94EB290E946A290E94B9
:1040D400EB290E9472290E94EB290E947D29EFADF1
:1040E4000E948429EFAD0E948B29EFAD0E94922992
:1040F400EFAD0E949929EFA70E94F0290E9464293C
:104104000E94F0290E94A4290E94F0290E94AA2951
:104114000E94F029E695E695E6950E94F5290E2E73
:10412400A0E035FCA1E0EA2FEE0FEE0FEE0FE02940
:10413400AE2FEFA9E2950E94FA29EFA90E94CA299D
:10414400EFA9E295EF70E695E170EA2BE8ABEFA9F1
:10415400E695E695E6950E946429EFA9E695E6952D
:104164000E94002AEFA90E94052AEFA90E94F529BE
:10417400AE2FEBA10E94BD29EBA10E940D2AEBA159
:104184000E94102AEBA1E695E170EA2BE9ABEBA1C2
:104194000E94DD29E8ADE2950E94002AE8AD0E9464
:1041A4007229E8AD0E94152AAE2FE8AD0E94BD2900
:1041B400E8AD0E940D2AE8ADE6950E94102AE8AD0C
:1041C400E170EA2BEAABEBA10E94E6290E94642984
:1041D400EAA10E94002AEAA10E94052AEAA1E69522
:1041E400E6950E94F529AE2FE0910103E2950E9425
:1041F4008429EBA1EE1FE0E0EE1F0E94FA29EAA158
:10420400E695E695E6950E94102AEAA1E295E1700A
:10421400EA2BEBABEAA10E94DD29E9ADE2950E940D
:10422400002AE9AD0E947229E9AD0E94152AAE2F39
:10423400EAAD0E94BD29EAAD0E940D2AEAADE695D9
:104244000E94102AEAADE170EA2BECABEAA10E94CD
:10425400E6290E946429EAADE2950E94002AEAADAB
:104264000E947229EAAD0E94152AAE2FE9AD0E9480
:10427400BD29E9AD0E940D2AE9ADE6950E94102AF8
:10428400E9ADE170EA2BEDAB33FE0DC051E05131E5
:1042940050F4E52FF0E0DE019596AE0FBF1FEFEF6F
:1042A400EC935F5FF4CF0E94192A5D3078F40E948A
:1042B4001F2AA2E5B8E00E94152CE17011F45D9864
:1042C40001C05D9A0E94262A5F5FEFCF0E942E2ACA
:1042D4005D3078F40E941F2AA0E3B8E00E94152CF8
:1042E400E17011F45D9801C05D9A0E94262A5F5F17
:1042F400EFCF0E942E2A5D3078F40E941F2AA2E09C
:10430400B8E00E94152CE17011F45D9801C05D9A2B
:104314000E94262A5F5FEFCF0E942E2A5D3078F438
:104324000E941F2AA6E0B8E00E94152CE17011F447
:104334005D9801C05D9A0E94262A5F5FEFCF0E94BC
:104344002E2A5A3098F45E9885E28A95F1F7E9E0CE
:10435400E51BA0E4B1E00E94152CE17011F45D9816
:1043640001C05D9A0E94262A5F5FEBCF41E0413194
:10437400E8F451E05930C0F45E9885E28A95F1F78B
:10438400E42FF0E0DE019596AE0FBF1FAC91E8E09C
:10439400E51B0E940D2CE17011F45D9801C05D9A3B
:1043A4000E94262A5F5FE6CF4F5FE1CF5D9A85E2E8
:1043B4008A95F1F7289A8DEC9AE00197F1F70E941B
:1043C4000A25A92DEAE00E94502C0E2AAB2DEAE022
:1043D4000E94502C0E2AAA2DEAE00E94502CE029BB
:1043E40029F0E0E0E0935103E0935203A82DE4E6C2
:1043F4000E94552C0E2EA0E0F099A1E00E943325D6
:1044040029F00E948E23F09AE89433F80C94B005B6
:10441400FFCFAA93E091C000E072E1F3E881E0935A
:10442400C60021960895A0913B03B0913C030895E2
:10443400A0919B03B0919C0380919D0390919E0356
:104444000895E0E0F0E061EE75E40E94862B0895A3
:10445400E0914703F09148030895662777270E9467
:10446400AE2A0E944E2D0895E0915303F091540317
:104474000895A091A303B091A4038091A503909102
:10448400A6030895E0E0F0E060E271E40895A091ED
:104494004703B09148030895E0E0F0E00E946C2CDB
:1044A4000895A0915303B09154030895E091CB0370
:1044B400F091CC036091CD037091CE0308950E94D6
:1044C400752AED93FC930895A091B703B091B803B6
:1044D4008091B9039091BA03E0E0F0E06AE774E4F4
:1044E4000E94382BDF01CB01ACCFA091B303B09174
:1044F400B4038091B5039091B6030895A091D703B6
:10450400B091D8038091D9039091DA030895E09192
:104514005F03F091600360916103709162030895F9
:10452400A4E6B0E080E090E00E94922CDF01CB0191
:10453400E091B303F091B4036091B5037091B603B5
:104544000E945D2D08950E94622D0E94E12A089523
:10455400E0915903F0915A030895E0935903F093BD
:104564005A030895A091D303B091D4038091D50345
:104574009091D6030895E093D303F093D40360930A
:10458400D5037093D6030895A0915F03B09160039F
:10459400809161039091620308950E94922CDF013F
:1045A400CB01E091D303F091D4036091D5037091D2
:1045B400D6030E945D2DC7CF0E94772AED93FC930A
:1045C4000895E0E0F0E061EE75E40E94382B089570
:1045D400A091BB03B091BC038091BD039091BE0335
:1045E4000895E0E0F0EC69E774EC0E94CB2B0895A9
:1045F400E7EEF3E0E0937503F09376030895E0911A
:10460400BB03F091BC036091BD037091BE03089598
:10461400E091BF03F091C0036091C1037091C203A4
:104624000895A0919F03B091A0038091A10390915C
:10463400A2030895E0939F03F093A0036093A10362
:104644007093A2030895A091A703B091A803809149
:10465400A9039091AA030895E0919F03F091A00308
:104664006091A1037091A2030895A091AF03B0914A
:10467400B0038091B1039091B2030895E0915B037C
:10468400F0915C0360915D0370915E030895E09383
:104694005B03F0935C0360935D0370935E03089582
:1046A400EDDFAFE3B0E00E94832D0895A0915B039A
:1046B400B0915C0380915D0390915E030895E0E006
:1046C400F0E060E070E00895DDDE0E94382B08958C
:1046D400E0E00E94552C0E2E0895A0917F03B09126
:1046E4008003809181039091820308950E22A0910A
:1046F4001E03ECE30E94502C0895A0915103B09145
:1047040052030895A0914F03B0915003C5CEE09198
:104714004F03F09150030895A4E6B0E00C94382AB6
:10472400E7EAE0937A00A4E00E948603EF2FF0E02A
:104734006E2EE7E2E0937A000895E7EAE0937A00C8
:10474400A3E00E948603EF2FF0E09E2EE7E2E093C1
:104754007A000895E7EAE0937A00A1E00E948603D4
:10476400EF2FF0E0BE2EE7E2E0937A000895E0E058
:10477400F0E00E948B2D0895EBE0E093E003E8EB7A
:10478400E093E1030895E8ECF0E0E0936503F0932F
:1047940066030895E0EDF7E0E0936703F0936803A0
:1047A4000895E0933F03F093400308950E942D2C55
:1047B4000E94AE2A0E944E2D089564DE0E94862B2C
:1047C4000895E0934503F09346030895E0935F034F
:1047D400F093600360936103709362030895E09320
:1047E4004F03F09350030895AAE0B0E00E94382AE2
:1047F400E7EAE0937A0008950E9486030E94222C3F
:104804000E941E2C08950E948603EF2FF0E0089565
:10481400E0938303F093840360938503709386038A
:104824000895E0913F03F09140030895E0918303DC
:10483400F091840360918503709186030895E7E203
:10484400E0937A008AE48A95F1F708958AE48A95D8
:10485400F1F7E7EAE0937A000895E0933503F093E3
:1048640036030895A0913503B09136030895FADF15
:10487400EAEFF0E00895F6DFEEE1F0E00E94662C46
:1048840008950E2EA52DE1E00E94552C0E22AA8932
:10489400E5E00E94502CE0210895AA89E5E00E94F9
:1048A400372C0E2EAE81ECE50895E0211E2EAA8948
:1048B400E7E00E94372C0E2EAE81ECE50895E0E08F
:1048C400E0933503E09336030895E6E00E94372C25
:1048D4000E2E0895AA2DEAE00E94502C0E2E089563
:1048E400A0E0F3FCA1E0E0E00E94372C0E22A22F0E
:1048F400E3E60895E0913503F09136030895F297C5
:10490400ADE7B0E00E948A2C0F010895F0E0DE01CB
:104914005796AE0FBF1FEC91F0E0D0010E94C22C5D
:104924009CDFA0DFA93CE0E0BE070895F0E0DE01D3
:104934005B96AE0FBF1FEC91F0E094DF0E948A2CCF
:10494400DF01E4E6F0E00E94C22C87CFE02FF0E024
:10495400DE015396AE0FBF1F0895A0917703B09167
:1049640078038091790390917A030895E8EEF3E057
:1049740060E070E00E94FF2CDF01CB01BBDF662703
:1049840077270895EC91F0E00E942D2CA8E0BCE478
:1049940081E090E00E94FF2CE0CFE0937703F09356
:1049A40078036093790370937A030895D6DFDECF9A
:1049B4000E94FC2BE5E0F0E060E070E00E94822CB5
:1049C40008950E94FC2BE4E1F0E060E070E00E94B6
:1049D4007A2C08950E94FC2BA431E0E0BE07E0E0AD
:1049E4008E07E0E09E070895E0917F03F091800335
:1049F4006091810370918203A0E5B4E180E090E0CE
:104A04000E94BD2CCACFE8EEF3E060E070E00895A8
:104A1400A62DEAE00E94502C0E2E0895A22FE3E664
:104A24000E94502C0895A0E0F0FCA1E0E0E00E9478
:104A3400372C0895E0E00E94552CE0210895A0E071
:104A440022FCA1E0E0E00E94372CE0210895A0912F
:104A54002D033ECEE0912C0340DEFF276627772707
:104A64000895E0E00E94372CE0210895EB85FC8551
:104A7400A0918303B0918403809185039091860370
:104A8400662777270E947A2C0E2EEAE0F0E060E099
:104A940070E00E94822C0895E0936503F09366030E
:104AA4000895C4DEAB85BC85882799270E94FC2B1A
:104AB4000895A630E0E0BE07E0E08E07E0E09E0740
:104AC4000895A0916503B09166030895E09165038C
:104AD400F09166030895EB85FC85A0918303B09162
:104AE4008403809185039091860366277727089530
:104AF400E32FA091C703B091C8038091C90390919B
:104B0400CA03FF27662777270E94AE2A0895AADEE4
:104B1400EAE00E94B22C0895E32FF0E0A091C703CD
:104B2400B091C8038091C9039091CA030E942D2CAF
:104B34000E94AE2A08CDA0916703B091680308953E
:104B44000E94322C0E945F2DFECCA32FBB27E09144
:104B5400C703F091C8036091C9037091CA03F0CFF1
:104B6400E0916703F091680308950E942D2C0E9440
:104B7400AE2A0895EAE0F0E00E94D52C6ECEE091D2
:104B84001403ABDDFF27662777270895E0936F03AF
:104B9400F09370030895E0911403F0E09EDD0E9409
:104BA4002D2C0E94FC2B08950E94B82CA0916F0319
:104BB400B09170030895E0916F03F091700308952C
:104BC400A0911403BB27E0917F03F09180036091CF
:104BD4008103709182030E94322C0E94FC2B089561
:104BE400A0E0F099A1E0E1E00E94372C7FCD0E22F5
:104BF400A22FE3E60E94372CE02108950E2EA09107
:104C04001E03ECE30E94502C0E2208950E948B2D6B
:104C1400A1E0B0E00C94382AE091B303F091B4031E
:104C24006091B5037091B603A3E3B0E00E94772AC4
:104C3400EDCFABE3B0E00E94772AE8CF89DCADE3A7
:104C4400B0E0E4CF0E94932DA1E0B0E00C94382AA8
:104C5400EAE00E94552C0E2E0895AB2DEAE00E9446
:104C6400502C0E2EA0E027FCA1E0E0E00E94372C9F
:104C74000E220895A0E0F2FCA1E0E0E00E94372CAF
:104C840008950E94372C0E2EA12FEBCEA92DEAE019
:104C94000E94502C0E2E0895E0E00E94372C0E2224
:104CA4000895E0910E03F0E0E75FFC4F0895E09172
:104CB4004503F09146030895E0913203EF5FE093DA
:104CC4003203E0913103A0913203EA1708950E9460
:104CD400502C0E2EA0E023FCA1E00895A0914503E2
:104CE400B09146030895A0915903B0915A030895D1
:104CF400E1E00E946B2DEA1B0E94BE2D0895A09155
:104D0400C703B091C8038091C9039091CA03089561
:104D1400E091C703F091C8036091C9037091CA037D
:104D24000895A0E0B0E080E09FE30E94E82A08959F
:104D3400E093B703F093B8036093B9037093BA0395
:104D44000895E6DFA3E7B3E037CCE0919703F09151
:104D540098036091990370919A030895EAE0F0E052
:104D64000E94C22C0895A0919703B091980380915A
:104D7400990390919A030895CADBD2CBE0939303ED
:104D8400F093940360939503709396030895F0E071
:104D9400EA0FFB1FE0934303F0934403AEE30C9448
:104DA4000B220E940B22A0E00C940B22E0914403FE
:104DB400AE2F0E940B22A09143030C940B22B0E06F
:104DC400E2E0F0E00E94D52C0895EAE0EEAFEFAF08
:104DD400DE01A05CBF4FEC930895DE01AF5BBF4FD3
:104DE400EC930895DE01AE5BBF4FEC930895DE01B2
:104DF400AD5BBF4FEC930895DE01AC5BBF4FEC930A
:104E04000895E9E0ECA3E0912E03E170EE0FE05881
:104E1400AE2FE0912E03E695E695E170EE0FEE0FCE
:104E2400EA0F0E2EA0E0F199A1E0EA2FEE0FEE0FAB
:104E3400EE0F0895ECA3E0912E03E170EE0FE0581D
:104E4400AE2FE0912E03E695E695E170EE0FEE0F9E
:104E5400EA0F0E2EA0E0F199A1E0EA2FEE0FEE0F7B
:104E6400EE0FE00DEBA30895E295E07FEE0FEE0F59
:104E74000895E0E020FCE1E0E0930103A0918703C2
:104E8400B09188038091890390918A030895A09139
:104E94008703B09188038091890390918A030895D0
:104EA400AA30E0E0BE07E0E08E07E0E09E07089548
:104EB40014DCEAE0F0E060E070E008950E94FF2C6A
:104EC400DF01CB01EAE0F0E060E070E00E94192D20
:104ED4000895E0917103F09172030E94012CDF01A7
:104EE400EAE0F0E00E94D52CE0937303F09374039E
:104EF4000895A0917303B09174030895FADFEAE072
:104F0400F0E008950E94D52CDF01EAE0F0E00E9471
:104F1400072D0895E4E6F0E060E070E00895B7DF5F
:104F2400EAE0F0E060E070E00895A0E020FCA1E099
:104F3400EA2FE295E07FABA1EA0FEBA30895A091DD
:104F44003D03B0913E030895FE01F6963D96BF01E0
:104F5400F6CFE8EEF3E00E94C22CDF01EAE0F0E0D5
:104F64000E94042DDB01EC930895FE01F6963E9613
:104F7400BF01E5CFE4E6F0E00E94C22CDF01EAE0E5
:104F8400F0E00E94042DDB01EC930895FE01F696F7
:104F94003F96BF01D4CFDF01EAE0F0E00E94042D88
:104FA400DB01EC9308950E94042DDB01EC9308953A
:104FB400BB27EAE0F0E00E94072D0895FE01F69673
:104FC4003A96BF010895EAE0F0E09CCFDB01EC9350
:104FD400FE01F69608950E94DA2CDF01CB01EAE087
:104FE400F0E060E070E00E94152D0895A031E7E242
:104FF400BE07E0E08E07E0E09E070895A83EE3E0E8
:10500400BE07E0E08E07E0E09E070895A436E0E0E6
:10501400BE07E0E08E07E0E09E07089547DBEAE084
:10502400F0E060E070E00895EFAFE4E7DE01A05C3B
:10503400BF4FEC930895DF01CB01E0E0F0E060E1C5
:1050440071EC0E94CB2B0895DF01CB01E0E0F0E08E
:1050540066EC72EC0E94CB2B0895DF01CB01C1CA30
:10506400A0918B03B0918C0380918D0390918E035A
:10507400089550DF23CFF4DFEAE0F0E060E070E071
:105084000895ECA1E058ECA3EEE3CECFE0916D03DC
:10509400F0916E030E94012CE0936D03F0936E0374
:1050A400089535DAA4E6B0E080E090E076CAA091F5
:1050B4006D03B0916E030895FE01F6963B96BF0111
:1050C4000895F5DFE0E1F7E21DCFFE01F6963C9688
:1050D400BF010895ECDFE8EEF3E014CFFE01F6968D
:1050E4003D96BF010895E3DFE4E6F0E00BCFFE0157
:1050F400F6963E96BF010895FE01F6963F96BF01CF
:10510400D6DFEAE0F0E00E94072DDB01EC9308957E
:10511400A0917503B09176030895FADFE4E6F0E018
:10512400F1CE3F96BF01F4DFEAE0F0E00E94072DE4
:10513400DB01EC930895DE01A05CBF4FEC9308956E
:10514400EAE0F0E00E94072D0895E985FA85F695D6
:10515400E79508950E94C22C1ECFDF01EAE0F0E03B
:105164000E94042D0895A0914903B0914A03089523
:10517400EAE0F0E00E94042D0895EAE0F0E013CFA5
:10518400ECA1E058ECA3E2E0EEAFEEE34DCFE9E3AF
:10519400D2DFE8E322CEE52FF0E0DE01D696AE0FB3
:1051A400BF1F08950E94372C0E2EAE8108950E94D1
:1051B400372C0E2AAE810895AD85BE85CFCDAE8144
:1051C400E5E0F0CFE3E10E94372CE0290895E72DD4
:1051D400F0E0DE015396AE0FBF1F0895A0917B034C
:1051E400B0917C0380917D0390917E030895EC91AE
:1051F400F0E00E942D2CA8E0BCE481E090E00E9445
:10520400FF2CECCFE0937B03F0937C0360937D034E
:1052140070937E030895E2DFA9CBEF85F8895DDA08
:10522400662777270E94BD2CEDCFA0918303B09110
:10523400840380918503909186030895EBAFF5DF95
:10524400EAE0F0E060E070E039CEECAFEEDFEAE0F7
:10525400F0E060E070E00E94192DEDAF08954ADBA4
:10526400F695E795FACAEAA3FDDAA436E0E0BE07AC
:105274000895F8DAE4E6F0E00E94C22C6ECFF2DA88
:105284006DCDF0DA75CFA0915703B091580308950E
:10529400E4E6F0E00E94C22C60CFE9E3EFAFE0E582
:1052A4004ADFEEE39ACDA0914103B0914203089501
:1052B400A0914D03B0914E030895A0913703B0918E
:1052C40038030895E170E795E0E0E795AE2F08957F
:1052D400E295EF70E695E170C7DDEA2BAE2F0895F5
:1052E400E295EF70E695E695E170E295E07FEE0FCA
:1052F400EA2BAE2F0895E295E170E295E07FEA2B68
:10530400AE2F0895E170EE0FEE0FEE0FEA2BAE2FE5
:105314000895E695E170EE0FEE0FEA2BAE2F089597
:10532400E695E695E170EE0FEA2BAE2F0895E6952B
:10533400E695E695E170EA2B0895FE01ED5BFF4FDB
:10534400E0810895E695E1708FDDEA2BAE2F089594
:10535400E695E695E170E295E07FEE0FEA2BAE2F3D
:105364000895E695E695E695E170E295E07FEA2BEF
:10537400AE2FECA10895E695E695E695C3CFE295A8
:10538400EF70E695E170EE0FEE0FEA2BAE2F089565
:10539400E295EF70E695E695E170EE0FEA2BAE2FFD
:1053A4000895FE01EE5BFF4FE0810895FE01EC5B82
:1053B400FF4FE0810895E295EF70E69583CFFE01FB
:1053C400EF5BFF4FE0810895E295EF70E695E69577
:1053D4000895FE01E05CFF4FE0810895FE01EB5B60
:1053E400FF4FE0810895E170E295E07FEA2B089594
:1053F400E170EE0FEE0FEA2BAE2F0895E17034DD6D
:10540400EA2BAE2F0895E695E170E295E07FEE0F6A
:10541400EA2BAE2F0895E695E695EACFE170EE0FFC
:10542400EA2BAE2F0895E295EF70E695DCCF28982D
:1054340085E28A95F1F751E008955E9885E28A95B0
:10544400F1F7ECE0E51B089585E28A95F1F75E9AA1
:1054540085E28A95F1F708955D9A85E28A95F1F7D8
:10546400289A84E191E00197F1F7E1CF109639F0A1
:105474008DEC9AE00197F1F7A8951197C9F7089573
:1054840030976040704009F070580895552342F4F5
:10549400503811F4E0FF04C03196691F791F6BF096
:1054A40050E8572711F45F93CFC05F3F31F0660F88
:1054B400000C57956795752F08955F9300200AF0A7
:1054C400CFC0C8C050E8192E1522880F991F952700
:1054D400550F879550E8072E0522660F771F75270D
:1054E400550F67950895689401C0E8945F93F2DFBF
:1054F400703818F07F3F08F4A7C056E1571BAAF490
:10550400519558300EF4593030F0EFEFFFEF6FEF54
:105514007FE777F91AC077275523B9F0EE0FFF1FFD
:10552400661F771F5A95D1F710C07727583028F097
:10553400EF2FF62F672F5850F9CF552331F076957A
:105544006795F795E7955A95D1F700200AF45BD152
:105554005F910895689401C0E8943097604070406A
:10556400B1F0002426F0772312F400944CD1172EC6
:105574007EE1112032F07A95EE0FFF1F661F111C99
:10558400F9CFEF2FF62F612D5F938ADF5F91089596
:105594004F93AF01FD01DA01AB01BC01CA01402DFB
:1055A400012C142E4F910895EA0FFB1F681F0895D4
:1055B400E095F0956095EF5FFF4F6F4F08955F930F
:1055C40081DF903871F150E8152604C05F937ADFCB
:1055D400903839F1703821F1572F591B2BF112F4FF
:1055E400D7DFFACF583118F0AA27BB2788275830BD
:1055F40028F0AB2FB82F88275850F9CF552329F01E
:105604008695B795A7955A95D9F7502D512572F0DF
:10561400CBDF38F46795F795E795739513F420C0BD
:10562400B7DF3EDF5F910895D8F7FBCFEA1BFB0B92
:10563400680B51F010F40094BBDF662392F3EE0F75
:10564400FF1F661F7A95CBF7EE27FF27662777277C
:105654005F910895EFEFFFEF6FE77FEF5F9108959C
:10566400EFEFFFEF6FE77FE75F9108955F932ADF26
:10567400703851F3903841F301240894791F23F4CE
:105684001CF300203AF3ECCF0F921F932F933F9318
:105694004F93112722279927689FA0018F9F302DB0
:1056A400410D591F6B9F300D411D591F8E9F27D0EF
:1056B400BF9F25D06A9F23D0BE9F1DD0AF9F1BD014
:1056C400AE9F110D291F391F491F591FE32FF42FB6
:1056D400652F522F4F913F912F911F910F90662369
:1056E4002AF0550FEE1FFF1F661F02C073954BF281
:1056F400CDDE5F910895100D211D391F02C0200DCC
:10570400311D491F591F08955F93DCDE703821F461
:1057140011200AF49FCFA4CF903809F495CF012427
:105724000894970B1BF4D4F30020F3CF792F1F9325
:105734002F933F934F931124112722273327442774
:10574400552790E2AE17BF078607410730F0AE1B1E
:10575400BF0B860B410B089401C08894551F221F70
:10576400331F111CAA1FBB1F881F441F9A9551F792
:10577400F901612D4F913F912F911F91662332F0D2
:10578400550FEE1FFF1F661F7A9543F27FDE5F9170
:10579400089599239AF0772342F0971748F029F453
:1057A400AE17BF07860720F031F0989488940895C7
:1057B4009894089408951894889408957723C2F7C8
:1057C400971798F3A9F7EA17FB07680788F399F383
:1057D400ECCFDFDFE1E009F008F0EE270895D9DF30
:1057E400E1E009F008F4EE270895EA0FFB1F681FB3
:1057F400791F0895AE1BBF0B860B970B0895F19587
:10580400E195F0400895F09560957095E195FF4F0E
:105814006F4F7F4F0895EE230E2EEA2F19F0E69571
:105824000A94E9F70895EE230E2EFD0121F0F69572
:10583400E7950A94E1F70895F695E795F695E795C7
:10584400F695E795F695E7950895FE2FFF0FFF0B64
:105854006F2F7F2F08956F2F660F660B762F089595
:105864008B2F880F880B982F0895EA17E1E009F031
:10587400EE270895EA17E1E009F4EE270895AE173C
:10588400E1E00CF4EE270895AE17E1E00CF0EE270A
:105894000895EA17E1E00CF0EE270895AE17E1E071
:1058A40008F0EE270895EA17E1E008F0EE270895DE
:1058B400EA17FB07E1E009F0EE270895AE17BF07EA
:1058C400E1E008F4EE270895AE17BF07E1E008F021
:1058D400EE270895EA17FB07E1E008F0EE270895A4
:1058E400EA17FB0768077907E1E009F0EE27089556
:1058F400AE17BF0786079707E1E00CF0EE2708957F
:10590400EA17FB0768077907E1E00CF0EE27089532
:10591400FA9FF02DEB9FF00DEA9FE02DF10D089515
:105924007A9F702D6B9F700DF89F700DE99F700D1D
:105934006A9F602D710DFB9F600D711DE89F600DC6
:10594400711D8827FA9FF02D610D781FEB9FF00DD4
:10595400611D781FEA9FE02DF10D681F781F0895DF
:105964006E2F6A9FF0016B9FF00D089574D0D0DF05
:105974000EF445DF08957DD0D3DF0EF444DF08959F
:105984000024112490E1AA0FBB1F001C111C0E1A45
:105994001F0A18F40E0E1F1E01C0A1609A9599F7F4
:1059A400FD01D001089557D0EBDF0EF428DF0895F0
:1059B4003F934F935F93002411244427552730E2EB
:1059C400AA0FBB1F881F991F001C111C441F551FC1
:1059D4000E1A1F0A460B570B28F40E0E1F1E461FE5
:1059E400571F01C0A1603A9559F7FD01BC01D001D0
:1059F400CA015F914F913F9108953BD0D9DF0EF4D6
:105A040002DF0895BDDFFD010895E894B7FF04C0E7
:105A1400A095B09511966894F7FDF1DEB1DFFD0114
:105A24000EF4EDDE0895C4DFFD01BC010895E89491
:105A340097FF09C0A095B09580959095AF5FBF4F33
:105A44008F4F9F4F689477FDDEDEB2DFFD01BC010E
:105A54000EF4D9DE0895E894F7FF02C0D0DE68940E
:105A6400B7FF06C0A095B095119600F8039400FA0C
:105A74000895E89477FF02C0C6DE689497FF0BC0D0
:105A84000024A095B095809590951196801D901D49
:105A940000F8039400FA0895ED93FD936D937C93BD
:105AA4000895A881B9818A819B810895E883F98347
:105AB4006A837B830895689401C0E89401D04DDD26
:105AC400182E862F612D192E972F712D1B2EBF2F67
:105AD400F12D1A2EAE2FE12D0895129602D0BF019A
:105AE4001297119602D0FE2F1197F999FECFFF93CA
:105AF400FFB7F894A1BDB2BDF89AE0B5FFBFFF911E
:105B0400089507D012960F01FB0103D0F0011297FC
:105B1400089507D01196EF93EF2F03D0EF911197CB
:105B24000895F99B02C0A895FCCF9FB7F894A1BD36
:105B3400B2BDF89A80B5E81719F0E0BDFA9AF99A5F
:105B44009FBF089500240E160F0606060706089543
:105B540000240A160B06089500240A160B060806EC
:105B640009060895EA17FB07680779070895AE1731
:105B7400BF07860797070895E894EE2309F0689411
:105B84000895AC0FBD1F05900D928A95E1F7089515
:00000001FF
